:100000002BC03AC039C038C037C036C035C034C044
:1000100033C032C031C04FC22FC02EC02DC02CC043
:100020002BC000003A00370000003B003800000001
:100030003900360001010101010101010202020241
:1000400001020408102040800402010800000000A2
:10005000000403020100000011241FBECFE5D1E01F
:10006000DEBFCDBF20E0A0E6B0E001C01D92A0370A
:10007000B207E1F76AD216C4C3CF813021F480B74A
:100080008F7780BF0895823019F480B78F7DF9CFC4
:10009000833021F48FB58F778FBD08958430E9F7D1
:1000A0008FB58F7DF9CFCF93DF93282F30E0F90103
:1000B000E45BFF4F8491F901E05CFF4FD491F901BB
:1000C000EC5CFF4FC491CC2399F08111D6DFEC2F6B
:1000D000F0E0EE0FFF1FE25DFF4FA591B491EC91B0
:1000E000ED2381E090E009F480E0DF91CF91089565
:1000F00080E090E0FACF1F93CF93DF93282F30E07A
:10010000F901E45BFF4F8491F901E05CFF4FD4916A
:10011000F901EC5CFF4FC491CC23A1F0162F8111A3
:10012000ACDFEC2FF0E0EE0FFF1FE85DFF4FA59175
:10013000B4918FB711110AC0F894EC91D095DE23D9
:10014000DC938FBFDF91CF911F910895F894EC91CC
:10015000DE2BF6CFCF93DF9390E0FC01E05CFF4F06
:1001600024918C5C9F4FFC0184918823C9F090E01E
:10017000880F991FFC01EE5DFF4FA591B491FC0122
:10018000E85DFF4FC591D49161110DC09FB7F89400
:100190008C91209582238C938881282328839FBF6C
:1001A000DF91CF910895623051F49FB7F8943C915C
:1001B000822F809583238C93E8812E2BEFCF8FB7EE
:1001C000F894EC912E2B2C938FBFEACF3FB7F89485
:1001D0008091650090916600A0916700B0916800E1
:1001E00022B708B600FE05C02F3F19F00196A11DE9
:1001F000B11D3FBFBA2FA92F982F8827BC01CD0171
:10020000620F711D811D911D43E0660F771F881FCE
:10021000991F4A95D1F70895CF92DF92EF92FF92FE
:10022000CF93DF936B017C01D1DFEB01CFDF6C1B40
:100230007D0B683E7340A0F0C114D104E104F104C9
:1002400039F4DF91CF91FF90EF90DF90CF90089538
:1002500081E0C81AD108E108F108C851DC4FE6CFA7
:10026000C114D104E104F10409F7EBCF2FB7F894DE
:1002700060916100709162008091630090916400D0
:100280002FBF0895CF93DF9382E00DDF892BB9F064
:1002900082E009DF892BD1F082E005DF019721F5AB
:1002A00087E001DF892B01F561E081E024DF82E056
:1002B000FADE0197E1F360E081E01DDF56C087E0E0
:1002C000F2DE892B29F7DF91CF91089587E0EBDEED
:1002D000019711F761E080E00EDF87E0E4DE01972F
:1002E000E1F360E080E0E9CF61E080E004DF88E0F6
:1002F000DADE892BC9F087E0D6DE892BA9F083E00E
:10030000D2DE0197B1F482E0CEDE019791F488E06D
:10031000CADE019771F487E0C6DE019751F468E206
:1003200070E080E090E004C06FE570E080E090E075
:1003300073DF61E081E0DFDED1E0C1E082E0B3DEC7
:10034000892B21F460E081E0D6DEC0E087E0ABDEFF
:10035000892B39F460E080E0CEDEC13031F4D0E0AA
:10036000EDCFC13059F3D13049F36CE271E080E058
:1003700090E0DF91CF9150CFCF93DF9388E093DE71
:10038000892B79F487E08FDE019759F483E08BDEC7
:10039000019739F482E087DE019719F4DF91CF915C
:1003A00071CF83E080DE892BB1F083E07CDE892B86
:1003B000C9F083E078DE019751F588E074DE892B7F
:1003C00031F561E081E097DE83E06DDE0197E1F3D6
:1003D00060E081E014C088E066DE892B31F7DF91B0
:1003E000CF91089588E05FDE019719F761E080E022
:1003F00082DE88E058DE0197E1F360E080E07BDE9A
:100400006CE271E080E090E0DF91CF9105CF61E098
:1004100080E071DE88E047DE892B21F087E043DE53
:10042000892B29F465E270E080E090E0F5DE61E080
:1004300081E061DE1BDFD1E0C1E083E034DE892BA7
:1004400021F460E081E057DEC0E088E02CDE892BFB
:1004500039F460E080E04FDEC13031F4D0E0EDCF20
:10046000C13059F3D13049F383E01DDE019741F6E5
:1004700061E081E040DE83E016DE0197E1F3A8CF82
:1004800087E011DE019729F488E00DDE019709F479
:10049000F9CE87E008DE892B09F46ECF88E003DE11
:1004A000892BB1F387E0FFDD892B21F488E0FBDDA8
:1004B000892B99F308951F920F920FB60F92112472
:1004C0002F933F938F939F93AF93BF93809161003E
:1004D00090916200A0916300B0916400309160003F
:1004E00026E0230F2D3768F129E8230F0396A11D7D
:1004F000B11D209360008093610090936200A093EF
:100500006300B09364008091650090916600A091B3
:100510006700B09168000196A11DB11D8093650030
:1005200090936600A0936700B0936800BF91AF916D
:100530009F918F913F912F910F900FBE0F901F9021
:1005400018950296A11DB11DD4CF81B781BF80B788
:10055000826080BF80B7816080BF83B7887F8360FF
:1005600083BF789489B7816089BF8EB5887F8EBD3F
:100570008FB581608FBD8FB58D7F8FBD8EB5877F25
:100580008EBD8EB58F7E8EBD8EB583608EBD86B1DD
:100590008877866886B9379A68E572E080E090E0EF
:1005A0003BDE62E08AE0D6DD62E089E0D3DD61E037
:1005B00081E0D0DD60E081E09EDD61E080E0CADDC9
:1005C00060E080E098DD60E083E0C4DD60E082E030
:1005D000C1DD60E088E0BEDD60E087E0BBDDD0E14A
:1005E00010E2C0916F008AE05EDD892B09F08DC0BA
:1005F000C46089E058DD892B09F089C08C2F8860A0
:10060000982F9670963031F486FD04C087FD02C0A5
:10061000807F8065982F9970993031F487FD04C0F0
:1006200086FD02C0807F806A82FF74C08160C82F0F
:1006300083FF72C0C2608AE036DD019729F489E049
:1006400032DD019709F4CF73C4FD68C0C0936F0019
:1006500080916F0085FF19C08F7D80936F0080911E
:100660006E008F7E69F402DE60936A0070936B0007
:1006700080936C0090936D0010936E00109269004F
:10068000809169008F5F80936900F0DD80906A003F
:1006900090906B00A0906C00B0906D0075016401AB
:1006A0002AEDC20E22E0D21EE11CF11CC616D706AE
:1006B000E806F90608F066C089288A288B2809F41C
:1006C00061C080916E00803109F0A0C08091690006
:1006D000813108F479C083E0E6DC0197C9F183E059
:1006E000E2DC019709F054C082E0DDDC019709F0FB
:1006F0004FC0C8DD68EC70E080E090E08DDD3CDE4E
:1007000068EE73E080E090E048C0CB7F72CF8C2F22
:10071000877F76CF8E7F8BCFCD7F8DCFCF7EC093DF
:100720006F0080916E008F7D69F4A0DD60936A0098
:1007300070936B0080936C0090936D00D0936E006B
:1007400010926900809169008F5F8093690080CF6B
:1007500082E0A9DC019719F688E0A5DC019709F091
:10076000BECF87E0A0DC019709F0B9CF10926E00F0
:1007700010926A0010926B0010926C0010926D0043
:100780001092690061E070E080E090E045DD29CFE3
:10079000F3DD68E572E080E090E03EDD61E080E05E
:1007A000AADC61E470E080E090E036DD61E081E0A9
:1007B000A2DC62E271E080E090E02EDD60E081E0AA
:1007C0009ADC60E080E01BC08630D8F05BDD61E041
:1007D00081E091DC83E067DC0197E1F360E081E098
:1007E0008ADC6AEF70E080E090E016DD61E081E095
:1007F00082DC82E058DC0197E1F360E081E07BDCA1
:10080000B5CF823008F4B2CF3BDEB0CF803209F0F2
:10081000ADCF80916900813158F134DD61E081E034
:100820006ADC83E040DC0197E1F360E081E063DCB7
:1008300061E081E060DC61E080E05DDC64EF71E05C
:1008400080E090E0E9DC8AE02EDC019721F489E089
:100850002ADC0197C1F360E081E04DDC60E080E0DC
:100860004ADC10DD6CE271E080E090E0D5DC7ECF08
:10087000863038F207DD61E080E03DDC88E013DCA3
:100880000197E1F360E080E036DC6AEF70E080E041
:1008900090E0C2DC61E080E02EDC87E004DC0197C0
:0808A000E1F38FCFF894FFCFC4
:00000001FF
